:020000040000fa
:080000000004040000000000f0
:020000040000fa
:1000080004180000081800000c1800001018000060
:1000180014180000bc180000bc180000bc18000030
:10002800181800001c1800002018000024180000f0
:10003800bc180000281800002c1800003018000018
:1000480034180000381800003c1800004018000060
:100058004418000048180000bc180000bc18000034
:100068004c180000501800005418000058180000e0
:100078005c180000bc180000bc180000bc18000088
:10008800bc18000060180000641800006818000020
:100098006c18000070180000741800007818000030
:1000a8007c18000080180000bc180000bc18000074
:1000b800bc18000084180000881800008c18000084
:1000c800bc18000090180000bc180000bc18000004
:1000d800bc18000094180000bc180000bc180000f0
:1000e800bc180000981800009c180000bc180000fc
:1000f800bc180000bc180000bc180000bc180000a8
:10010800bc180000bc180000bc180000bc18000097
:10011800bc180000bc180000a0180000bc180000a3
:10012800bc180000a4180000a8180000ac180000b3
:10013800bc180000bc180000bc180000bc18000067
:10014800b0180000bc180000bc180000bc18000063
:10015800bc180000b4180000bc180000bc1800004f
:10016800bc180000bc180000bc180000bc18000037
:10017800bc180000bc180000b8180000bc1800002b
:10018800bc180000bc180000bc180000bc18000017
:10019800bc180000bc180000bc180000bc18000007
:1001a800bc180000bc180000bc180000bc180000f7
:1001b800bc180000bc180000bc180000bc180000e7
:1001c800bc180000bc180000bc180000bc180000d7
:1001d800bc180000bc180000bc180000bc180000c7
:1001e800bc180000bc180000bc180000bc180000b7
:0801f800bc180000bc18000057
:020000040000fa
:100208009a0400009a0400009a0400009a0400006e
:100218009a0400009a0400009a0400009a0400005e
:100228009a0400009a0400009a0400009a0400004e
:100238009a0400009a0400009a0400009a0400003e
:100248009a0400009a0400009a0400009a0400002e
:100258009a0400009a0400009a0400009a0400001e
:100268009a0400009a0400009a0400009a0400000e
:100278009a0400009a0400009a0400009a040000fe
:100288009a0400009a0400009a0400009a040000ee
:100298009a0400009a0400009a0400009a040000de
:1002a8009a0400009a0400009a0400009a040000ce
:1002b8009a0400009a0400009a0400009a040000be
:1002c8009a0400009a0400009a0400009a040000ae
:1002d8009a0400009a0400009a0400009a0400009e
:1002e8009a0400009a0400009a0400009a0400008e
:1002f8009a0400009a0400009a0400009a0400007e
:100308009a0400009a0400009a0400009a0400006d
:100318009a0400009a0400009a0400009a0400005d
:100328009a0400009a0400009a0400009a0400004d
:100338009a0400009a0400009a0400009a0400003d
:100348009a0400009a0400009a0400009a0400002d
:100358009a0400009a0400009a0400009a0400001d
:100368009a0400009a0400009a0400009a0400000d
:100378009a0400009a040000bc1600009a040000c9
:100388009a0400009a0400009a0400009a040000ed
:100398009a0400009a0400009a0400009a040000dd
:1003a8009a0400009a0400009a0400009a040000cd
:1003b8009a0400009a0400009a0400009a040000bd
:1003c8009a0400009a0400009a0400009a040000ad
:1003d8009a0400009a0400009a0400009a0400009d
:1003e8009a0400009a0400009a0400009a0400008d
:0803f8009a0400009a040000c1
:020000040000fa
:100800000fa220000e7f22000e01880000000000d1
:10081000000020000000e000020032000001200083
:10082000200288000c000700007221000100200057
:1008300011000700000020000000e000020032006c
:100840000000020000000000481602000000000046
:100850000040da000000fe004440a900000c200027
:100860000000e0000300320000002000a00188002a
:100870004440a80000000600910188008000780034
:100880000000eb0015003700e280400032a0b40009
:100890009101ba00e280400032a0b4009102ba0097
:1008a000e280400032a0b4000002eb00472bde00e3
:1008b000f507b200602ce10004003a000059eb009b
:1008c0008301e900fdff3e00040037006128e100dc
:1008d000010032000082eb00040007001101ba00a1
:1008e0000200e000e8ff3a00000006003159ba00bb
:1008f0008301e9000c0032002159ba008301e900ac
:10090000080032000400e00003003a00e2804000ea
:1009100032a0b400f5ff370011d9ba008301e90015
:10092000faff3a008100e800e180400032a0b40004
:10093000000006000040da000000fe00000278001f
:1009400002003700015a78000201e900e00f51006f
:08095000fcff3a000000060064
:020000040000fa
:100958001201000010010000000000000008000063
:10096800d80400003c000000020000000102000062
:100978000001000009020000290000000101000038
:1009880000c000003209000004000000000200005e
:100998000300000000000000092100001101000010
:1009a80000010000221d0000000700000581000072
:1009b80003400000000100000705000001030000db
:1009c80040000000010000000403000009040000ca
:1009d800340300004d0000006900000063000000bf
:1009e800720000006f000000630000006800000053
:1009f80069000000700000002000000054000000a2
:100a08006500000063000000680000006e00000040
:100a18006f0000006c0000006f000000670000001d
:100a28007900000020000000490000006e0000006e
:100a3800630000002e00000026030000550000009f
:100a480053000000420000002000000048000000a1
:100a5800490000004400000020000000420000009f
:100a68006f0000006f000000740000006c000000c0
:100a78006f000000610000006400000065000000d5
:100a88007200000006000000ff09000001a100003c
:100a9800011900000129000040150000002600008f
:100aa800ff0000007508000095400000810000006c
:100ab800190100002940000091000000c00000005a
:100ac800be840000e8840000ec840000208500005b
:020000040000fa
:100ad8000080fb008182fb0000024000048242008b
:100ae8004322dd0005a020000502420014f0a10009
:100af800e0cf500004003a0000004000a59220001a
:100b0800843278000300370000004000e59220009e
:100b18008432780014e0a1006402420014e0a000ce
:100b280000000600e548800084c0b300e78f52004b
:100b380011003e00e448800085932000954278002b
:100b4800e0cf520005003a0015c0b3008002fd0056
:100b580038e9b7008002fd000700370085932000c0
:100b680095427800e1cf520003003a0025c0b30057
:100b78000500780038e9b7000480fb001c29b5009f
:100b880075498000844a7800e5942000d54988009a
:100b98001a09ab0003003200e04f52000b003a0084
:100ba80000000600e04f52000f003200c5488000e8
:100bb800d6498000355b7800d6498800c54888004a
:100bc8000442e900f9ff3a0000000600c548800029
:100bd800d6498000355b7800d6498800c54888002a
:100be8000442e900f9ff3a0000000600659420007d
:100bf8009542780004c8b30084cf520038003a0008
:100c080004ccb3000002fd001ae9b7000002fd00a1
:100c18009494200014427800e24f520009003200f8
:100c2800e34f52001b003200e14f52002b003a0004
:100c3800c44a2800c448880024012000e4488800e9
:100c4800000006008494200014427800e04f52000f
:100c58000e003a0084942000144278000482fb00bd
:100c68000402420045562800e5027a00c54888007b
:100c7800c4488000244090001ce9b700c4488000a4
:100c8800344090001de9b700000006001a69ef0023
:100c9800000006008494200014427800e24f5200bd
:100ca8000c003e0084942000144278000482fb006b
:100cb8000402420065562800e5027a00c54888000b
:100cc800c4488000144278000482fb00e44888008d
:100cd800000006001a69ef00000006001a69ef001c
:100ce800000006000042eb000002fd004ee9b700dc
:100cf8004fe9b7000002fd00649420001442780018
:100d08007f026200e10f52000b003200e20f520036
:100d18000b003200e00f520023003a001ae9a80045
:100d2800e491200014427800e04f52001e00320087
:100d38004e29a8001c0037001ae9a8001a0037003d
:100d48001ae9a800a494200014427800e04f520049
:100d580007003500a4942000144278006f02620056
:100d680004024200a5922000e5027a00060037003e
:100d7800a4942000144278006f026200040242002a
:100d8800e5922000e5027a000440280095026200fe
:100d9800848f520004003a0014c0b3000002fd0022
:100da8004ee9b7000002fd0004082000d548800085
:100db8000502620007003200e4942000c44888005d
:100dc8001a09a80024c0b3000002fd001ce9b700fe
:100dd8000002fd0000000600aa24ab00110032004a
:100de800a44980001443900005c8b300854f530000
:100df8000b003a00754980001543900045c8b300c0
:100e0800854f530006003a00c5c0b300154298004c
:100e1800a4498000944290000574a00015429800ef
:100e2800aa24a90004082000542488000000060011
:100e3800881f780074498000140478004e44de004e
:100e4800614464002e49aa0004498000e80f52005a
:100e58000c003a008494200014427800f407b20091
:100e6800b4248800b4248000e00f5200030032004c
:100e780004012000044988000200370044002000d3
:100e8800044988009493200014427800e14f5200ee
:100e980022003a00e5942000744980001502980069
:100ea80020ff07008493200014427800e24f52008c
:100eb80008003a0045c0b300744980001542980004
:100ec80074498000944290000574a000154298006f
:100ed80028003700e04f540008003a0085c4b300ea
:100ee800744980001542980074498000944290002b
:100ef8000574a000154298001e00370085c0b30095
:100f0800744980001542980074498000944290000a
:100f18000574a0001542980016003700549220006e
:100f280014427800e04f520011003d0084922000e6
:100f3800144278000482fb009592200095427800c4
:100f4800c82add00050272000800320084922000e1
:100f5800144278000482fb009592200095427800a4
:100f6800c82add00050272000400010025e9a90075
:100f78003969ef004f047800000006001f69ef0090
:100f88000001eb008000eb00400720004907070044
:100f98008284a900040120000424880000000600bf
:100fa8008284a800040120005424880014c0b300df
:100fb800040078001fe9b7000001eb008000eb0097
:100fc800500720003b0737000200fa00881f78000e
:100fd8008494200014427800e14f52000f003a0038
:100fe80064942000144278007f4262000b003a00ab
:100ff8001ae9a8007494200014427800e34f5200c4
:1010080005003a0014c0b3000002fd001ee9b70055
:101018000002fd00010037001e69ef0084942000e3
:1010280014427800e04f5200ad003a00649420006a
:10103800144278007f426200e24f5200a8003a0052
:10104800a4942000144278006f426200a400320089
:10105800a4942000144278006f026200e10f52004d
:101068009f003c000549800004022000848f520044
:101078009b003a001ae9a800a494200014427800c2
:10108800e04f52000d003500a4942000144278006f
:101098006f02620004024200a5922000e5027a0075
:1010a800e5bf9f00a4942000144278006f026200fc
:1010b8001594200065447a000c003700a4942000a1
:1010c800144278006f02620004024200e592200098
:1010d800e5027a00e5bf9f00a4942000144278003e
:1010e8006f026200f593200065447a006142640053
:1010f80004003a004ffa97000424a100c4ff9f009f
:1011080003003700cffa97000524a000c5ff9f0011
:10111800a494200014427800e04f520008003500e3
:10112800a4942000144278006f0262000402420076
:10113800a59220006fbb970086327a00070037001f
:10114800a4942000144278006f0262000402420056
:10115800e59220006fbb970086327a0074942000d5
:1011680014427800e34f52001d003a006fba97000e
:101178008002eb00948f120013003d00a49420001d
:1011880014427800e04f520008003500a594200072
:1011980095427800ef8262001694200066c27a00b9
:1011a8000410a00004f37a0007003700a59420007b
:1011b80095427800ef826200f693200066c27a00ba
:1011c8000410a00004f37a006fba9700144390004b
:1011d80045c8b300854273001542980040003700a7
:1011e8004ffb97000624a200c6ff9f00efb89700a8
:1011f8000002eb00910f120008003d001142900020
:101208000474a1000464a000944098002200200007
:1012180050002000a7060700030037001142900085
:101228000464a00094409800cffa97000524a20017
:10123800c5ff9f006244640004003a006fba97003b
:101248000003eb00940f13001b003d00a494200042
:1012580014427800e04f520008003500a5942000a1
:1012680095427800ef8262001694200066c27a00e8
:101278000410a10004f37a0007003700a5942000a9
:1012880095427800ef826200f693200066c27a00e9
:101298000410a10004f37a00efb8970011429000ff
:1012a800b443b2009440980022002000500020006f
:1012b800800607000300370094429000b543b2004f
:1012c80015429800a4942000144278006f0262002e
:1012d80004024200a54a2000050242001414a1009d
:1012e8004f0478000080fa0000000600889fbe00c6
:1012f8001ae9a8000004eb006825880009a020006e
:1013080002022000880078000900780089fd0700a3
:101318009424a8000004fd003fe9b70041e9b700a4
:1013280040e9b70042e9b70032e9b7000004fd0020
:101338009424a9006882440074498800a949880057
:10134800b949880048c9bf0022e9b70024922000a3
:1013580014427800e04f520003003a0004012000d4
:10136800044988000600370012002000219220005e
:10137800100020004f0607000402200004498800de
:101388004f04be0000000600649420001442780058
:101398000446b2003f003a007494200014427800da
:1013a8000482fb0005002000eb0f5200e08f5a007a
:1013b80038003e00046001001a0037001a003700a8
:1013c80034003700180037003200370006003700b5
:1013d800090037002b0037000900370007003700e5
:1013e800120037001e0037001ae9a8008400200008
:1013f8000449880000000600fcfd3700bbff3700e9
:1014080024922000c44888001a09a80014c0b30018
:101418000002fd001ce9b7000002fd001ae9a8005f
:10142800000006002ffe3700e7fe3700a5942000d5
:10143800954278008582fb002493200004824200b4
:10144800c44888001a09a80014c0b3000002fd00af
:101458001ce9b7000002fd001ae9a8000000060018
:101468001ae9a800a4942000144278000482fb0022
:1014780025932000869420001643780086727a000f
:10148800000006000001eb008000eb0020002000b7
:1014980008060700000006009ec0a9000082eb00b5
:1014a80074248800542488000003eb005625880023
:1014b80066258800240020003425880046258800f9
:1014c8008644a900f4092000842488006424880044
:1014d8008804a80004a020004822de00c424880054
:1014e8006022b800045088001550880024508800f5
:1014f8003550880044508800555088006450880052
:10150800755088008450880095508800a450880041
:10151800b5508800c4508800d5508800e450880031
:10152800f55088009424a800b624880094a4a90043
:101538009424a9005424800068026200860f520097
:1015480013003200860020000042eb005624880079
:101558000002fd001ae9b70025e9b7000002fd0006
:1015680065922000954278000002fd0026e9b70048
:101578000002fd0075922000954278000002fd00ef
:1015880027e9b7000002fd008a64ab00efff3a00cc
:1015980014c0b3000002fd0044e9b70045e9b700f4
:1015a8000002fd000042eb000002fd0016e9b70052
:1015b80014e9b7001fe9b7000002fd008002eb0044
:1015c800554988000002fd003fe9b70041e9b7002e
:1015d8000002fd0085498800654988000002fd0079
:1015e80040e9b70042e9b7000002fd0086a02000ec
:1015f80076498800d6002000562588006694200089
:101608001650880086c0b3000600780000eab700cc
:1016180046c0b3000600780001eab70001eaa80056
:101628000400780022e9b700054988000000060098
:10163800889fbe008a1f78008044780001447800a3
:101648000885fb0068026500030032008040eb005b
:10165800094078001efd070064056500030032009c
:1016680011c0b3000940780019fd07008984fb0008
:1016780089844400a44a200008f27c004f057800c1
:101688004f04be0000000600e0cf50000500320005
:101698000082fb0004024200e592200065027a0005
:1016a800040037000082fb0004024200a5922000db
:1016b80065027a008002eb00850f52001a003200a2
:1016c80012029800034a7800944290000544b20040
:1016d80015429800944290000534a00015429800e5
:1016e800944290000574a00015429800e0cf500085
:1016f800070032000080fb0000004000e592200057
:10170800050040001024a20084027800060037007b
:101718000080fb0000004000a5922000050040006a
:101728001024a2008402780005007800000006005a
:10173800e04f500015003a0085c0b300b44980005e
:10174800054a7800b4498000659420001502980085
:10175800c5c0b30015429800b449800014439000f6
:1017680005c8b300054373001642980046c0b3008d
:101778007449800016429800744980001443900010
:101788008542730015429800000006000182fb00a4
:101798000080fb0000004000000242004322dd0000
:1017a80006a02000860342001740900045c8b300f9
:1017b800054070009043980064024200060242000f
:1017c80014439000854273001542980000000600fb
:1017d80005022000a42480008482620018003200e0
:1017e8000082fb0004024200e592200004824200cd
:1017f800140378001601be00000420000100200038
:101808000201600003002000028bbe001403780070
:101818001601be00001b6900019369001424a20090
:1018280014037800964390000744b20017439800c9
:10183800140278001443900080426b00154298000f
:10184800000006000002eb00a4248800642488003d
:10185800044988000000060004498000e00f520097
:1018680011003a00a4248800642488002500200080
:1018780035258800442588008644a900f4092000fd
:1018880084248800642488009ec0a8009404ab00c7
:1018980003003a009404a8009404ab00fdff320052
:1018a8001400200004498800000006004494200029
:1018b80014427800e04f520035003a0014c0b300db
:1018c8000002fd0044e9b7000002fd005494200026
:1018d80014427800e04f52002d003a0014c0b300c3
:1018e8000002fd0045e9b7000002fd0094932000c6
:1018f80014427800e24f52000a003a00744980000e
:10190800004aeb0085c4b300744980001542980072
:1019180074498000944290000574a0001542980014
:10192800000006009493200014427800e14f520012
:1019380017003a003e69ef0084c0b300a549800053
:10194800844a7800a5498000669420009602980091
:1019580047c0b30097429800a749800017409000fd
:1019680005c8b300054070009043980017c0b30045
:101978008003fd003ee9b7008003fd00b749800001
:10198800844b7800b44980001602980015429800ec
:1019980000000600a4498000944378006492200067
:1019a800144278000482fb0075922000954278006a
:1019b800c82add00050272008782fb00848f52006e
:1019c8000400360067922000974378007492200044
:1019d8001442780064922000144278000482fb00cc
:1019e8007592200095427800c82add000502720031
:1019f8008782fb000502520065922000954278001c
:101a08000002fd0026e9b7000002fd004822de00c2
:101a180075922000954278000002fd0027e9b70082
:101a28000002fd00e0cf5300180032008002eb00f6
:101a380034922000144278000482fb004692200071
:101a4800164378004833dd0006027200e694200051
:101a580066da7a0036922000164378000002fd000c
:101a680023e9b7000002fd004822de00469220006c
:101a7800164378000002fd0024e9b7000002fd00cb
:101a88008502e80085cf5300e9ff3e0064922000fc
:101a9800144278000482fb00759220009542780079
:101aa800c82add00050272001a00320085c0b300a2
:101ab800b4498000054a7800e5942000b4498000c4
:101ac8001502980004002400a54980001502620050
:101ad80008003a0085c4b300b44980001542980054
:101ae800b4498000944290000574a0001542980003
:101af8000000060085c0b300b44980001542980074
:101b0800b4498000944290000574a00015429800e2
:101b18000000060085c0b300b4498000054a78007b
:101b2800b4498000659420001502980045c0b300b0
:101b380015429800b4498000944290000574a000b2
:101b48001542980084922000144278000482fb0019
:101b58009592200095427800c82add00050272009f
:101b68000800320084922000144278000482fb00ae
:101b78009592200095427800c82add00050272007f
:101b88000400010025e9a9005491200014427800be
:101b9800e04f520001003a0044ff07000000060031
:101ba8009493200014427800e24f520001003a005a
:101bb80078ff37003969ef00e49320001442780079
:101bc800e04f52000d003a0085c0b300b4498000d0
:101bd800054a7800b44980006594200015029800f1
:101be800c5c0b30015429800b449800094429000e3
:101bf8000574a00015429800000006003e69ef0039
:101c0800000006000042eb000002fd0016e9b700e4
:101c180014e9b7000002fd009493200014427800f4
:101c2800e24f52000d003a0085c0b300b44980006d
:101c3800054a7800b4498000e59420001502980010
:101c480085c4b30015429800b449800094429000be
:101c58000574a0001542980000000600c5942000f5
:101c6800954278008582fb00d494200014427800c5
:101c78004822dd0084827200e4488000848f52008c
:101c880008003100c4942000144278000482fb004c
:101c9800d594200095427800c82add00050272001c
:101ca800e44888009ffb0700e59420007449800001
:101cb8001502980085c4b300744980001542980045
:101cc80074498000944290000574a0001542980061
:101cd8000000060094a4a90004082000d54880004c
:101ce8000502620028003a0054922000144278004d
:101cf800e04f52000f003d0024c0b3000002fd0079
:101d080039e9b7000002fd00449120001442780030
:101d1800e04f520001003a00baff07000042eb0012
:101d28000002fd0045e9b70044e9b7000002fd00e4
:101d38000000060085c0b300b4498000054a780059
:101d4800b44980006594200015029800c5c0b3000e
:101d580015429800b44980001443900005c8b300a8
:101d6800054373001642980046c0b30074498000ca
:101d7800164298007449800014439000854273000d
:101d88001542980000000600649420001442780070
:101d9800e04f520013003d0014c0b3000002fd00e4
:101da80039e9b7000002fd00649120001442780070
:101db800e04f520001003a0092ff07000042eb009a
:101dc8000002fd0045e9b70044e9b7000002fd0044
:101dd8005491200014427800e04f52001b003a0052
:101de800b2fe370024c0b3000002fd0039e9b70095
:101df8000002fd0085c0b300b4498000054a7800a0
:101e0800b4498000659420001502980045c0b300cd
:101e180015429800b4498000944290000574a000cf
:101e2800154298000042eb000002fd0045e9b700aa
:101e380044e9b7000002fd005491200014427800e4
:101e4800e04f520001003a0098fe0700000006002b
:101e5800881f78000042eb000002fd0038e9b70057
:101e680015e9b70016e9b70014e9b7003ee9b7006d
:101e78000002fd000002fd0039e9b7000002fd0084
:101e880075498000154390000674a1009642980099
:101e9800e59220001524a200764980009643900020
:101ea8000774a100174398001524a200b5498000c3
:101eb800154390000674a100964298000002fd00a8
:101ec8001ae9b7000002fd000004eb00e8488800aa
:101ed8000002fd0025e9b7000002fd006592200020
:101ee800954278000002fd0026e9b7000002fd00d7
:101ef80075922000954278000002fd0027e9b7009e
:101f08000002fd0020fd0700080178008800780025
:101f180030002000670307006eff07004f047800b9
:101f280000000600d4c2b3000002fd0043e9b70078
:101f38000002fd00c493200014427800b40fb200e0
:101f48001f003a00c493200014427800c40fb20066
:101f580005a0200005024200a4498800b449880071
:101f6800844278000524a2008002fd0036e9b7000b
:101f78008002fd0006c0230014036300054023000f
:101f8800850f53000d003a00659420000500780085
:101f9800e883420014039000965a780014039000d6
:101fa8000603e80016029800878f5200f9ff3a00ee
:101fb800a449800010029800a5ff3700f8fe3700fa
:101fc800c493200014427800b40fb200e80f520006
:101fd80001003a0096fb070000000600889fbe003b
:101fe8008a1f780004498000e10f520009003a0076
:101ff80004042000a52480000502620005003a00c0
:102008008aa4ef008c04a8008c84a8002400200077
:10201800044988008084ab00050032008284ab004c
:10202800030032000401200004248800d3fb0700c9
:102038008824ab00020032008ec0a9007d00370062
:102048008a04ab00080032008c04ab0006003200a2
:1020580011fd07009ec0a800440020000449880024
:1020680014002000542488008a84ab000500320044
:102078008c84ab0003003200c9fb07000401200078
:10208800542488008a44ab00120032008c44ab0010
:1020980004003200120020008000eb00300720000e
:1020a80004030700440020005424880034942000ce
:1020b80014427800e04f5200010032004369ed00fd
:1020c8003494200014427800e04f520001003a0096
:1020d800f6fd070004082000552480000502620070
:1020e8000500320004082000652480000502620013
:1020f8000100320038fb07008a24ab0009003200d7
:102108008c24ab0007003200120020008000eb0096
:10211800f0ff2700e70207008ea4ef00240020004c
:102128005424880004498000e30f520002003e0056
:102138008ec0a9003f0037008c64ab003c00320021
:10214800542480006802620048c0b3008a0020005e
:10215800e9cfb30003003a00350037008a64ab00ca
:1021680033003200942480000002fd003ce9b700ef
:102178000002fd00c4932000144278000482fb0092
:102188004422de000002fd003de9b7000002fd0028
:102198005a248800c49320001442780068426200e0
:1021a8000c003a00d4932000144278000482fb000b
:1021b8001594200065437a00614363000604a20079
:1021c800e5437a0089c3630006c3730086727a0008
:1021d8000b003700d4932000144278000482fb00df
:1021e800f593200065437a00614363000604a2006a
:1021f800e5437a0089c3630006c3730086727a00d8
:10220800d493200014427800e04f520002003a00b4
:1022180044ff0700040037000001eb00c1932000d1
:1022280020072000a30207000844e900cbff3a007a
:102238008ec0a9004f0578004f04be0000000600bc
:10224800889fbe008004eb00094088001940880080
:1022580094c2b30004007800c4e8b70004802a00e0
:1022680034468800c828ef0018c0b300080078007a
:1022780012e9b70009007800cae8b7000ea9ef0014
:1022880010a9ef00090078000ce9b700d1c1b3002c
:1022980008407800e6fc070003c4b3004288200029
:1022a8008940780008407800f7fc07000040880063
:1022b8004f04be0000000600b68c200016437800cc
:1022c8000683fb00070020004a3add00c632de0024
:1022d800850272004a32dd0026042400063b88008d
:1022e8000583fb00960188000083eb00060abb000b
:1022f8001000fc0054052000343b8800a40a20008c
:10230800343b880061e7a8000000000000000000de
:1023180005002800063b800006826200fdff3a00a7
:102328000000060034002400043b88000cc9bf00ec
:102338001c003200c58c2000040028000080fb002f
:102348000100200076488000874880000000530084
:1023580081805b00910188001508bb00150390007f
:102368000688bb001000fc0056052000363b88009c
:10237800a60a2000363b880061e7a800000000009c
:1023880000000000073b800007036200fdff3a00e1
:102398000cc9ed000ce9b700e4824200e04f5000a0
:1023a800e6ff3a0061c7a900000006009501800019
:1023b80091018800000278001483ba008600780032
:1023c8001400ba009501880000000600889fbe002e
:1023d8008a9fbe00a48c200014427800e04f52006f
:1023e80027003a0014408000e00f5200030032003a
:1023f8000000eb00940f10009201350004408000ab
:10240800e00f520005003a00348820003580200093
:102418000604200004034300040037008002eb0098
:10242800948f1200f8ff3d0086013700d46a7800c7
:10243800860f5200fdff3a0003c4b3004288200013
:102448008040eb0010c0b3008ffc070000408800fc
:1024580014c0b3000002fd00cae8b7000002fd0086
:102468003484200006042000040343008042eb006b
:10247800056a7800860f5200fdff3a0071013700a7
:1024880044802000144278000482fb0005002000ec
:1024980062025200e0825a00e60f5200e08f5a00b2
:1024a80068013e0004600100060037006200370042
:1024b8007a00370091003700f0003700f400370049
:1024c8005a01370024c0b3000002fd0044e8b700f9
:1024d8000002fd0085c3b3008002fd0045e8b70097
:1024e8008002fd000002fd0046e8b7000002fd0082
:1024f80014c0b3000002fd0047e8b7000002fd0069
:102508000042eb000002fd0048e8b7000002fd00b1
:1025180085c1b3008002fd0049e8b7008002fd00d4
:102528000002fd004ae8b7004be8b7000002fd00d2
:1025380004802e00f5ff2f003646800047468000b5
:102548000602420087824a000002fd004ce8b700fc
:102558000002fd004823de000003fd004de8b7003f
:102568000003fd008002fd004ee8b7008002fd0078
:10257800482ade000002fd004fe8b7000002fd0017
:1025880050e8ef002491200014427800e04f5200f8
:102598001b003a0034c0b3000002fd0050e8b70049
:1025a8000002fd000042eb0085cfb3008002fd0071
:1025b80051e8b7008002fd00b5cab3008002fd00f3
:1025c80052e8b7008002fd000002fd0053e8b700a2
:1025d80054e8b7000002fd0085c0b3008002fd008a
:1025e80055e8b7008002fd000002fd0056e8b7007c
:1025f80057e8b70058e8b7000002fd0059e8ef00b7
:1026080014408000e00f5200030032008003eb000a
:10261800948f13000b01350003c4b30042842000db
:1026280011c0b3000140780017fc07001040880073
:10263800ca68ef0003013700548020001442780074
:10264800e04f520008003a00a4c2b300040078002a
:10265800c4e8b70080bf2a0030468800c828ef00c9
:102668001269ef000b00370094c2b3000002fd00ae
:10267800c4e8b7000002fd0004802a003446880040
:10268800c828ef0014c0b3000002fd0012e9b7002b
:102698000002fd00ca68ef00ea00370064c0b3001a
:1026a8000002fd00cbe8b7000002fd00448c2000ca
:1026b800144278000482fb000402e800e60f52008e
:1026c8000b003400fcfe070044fe0700cb48ec007a
:1026d800cbe8b7000080fb00448c2000144278004f
:1026e8000482fb000402e800840f5000f5ff350067
:1026f80061c7a900ca68ef00d2003700744880009b
:1027080085488000e10f4200e08f4a0012003a003d
:1027180056802000164378000683fb00678020005f
:1027280097437800c83bdd00060278000702720074
:1027380076802000164378000683fb0087802000ff
:1027480097437800c83bdd008602780087827200d4
:102758007448880085488800568020001643780011
:102768000683fb006780200097437800c83bdd00a4
:10277800060278000702720076802000164378006f
:102788000683fb008780200097437800c83bdd0064
:102798008602780087827200764880008748800029
:1027a800860f5200878f5a0032003a00948020002a
:1027b80014427800e14f52002e0036000044eb002e
:1027c800c98c20008a032000c5902000954278001b
:1027d8000583fb00860343000482fb0004025500c6
:1027e80026002000110009000602d8000002780027
:1027f8000880fb000002420064024200040242001a
:102808004680200066407a000080fb0004024300f6
:10281800144290004822dd00040070000002780095
:1028280084b47b000542e8000002fd000ce9b70013
:102838000002fd007648800087488000610343005d
:10284800e0834b007648880087488800fc4f520098
:1028580001003a00b3fe07000844e8009480200015
:10286800144278008482fb008502d100854f540011
:10287800d5ff3900ca68ef0072003700a9fe0700cb
:102888000ea9ef0010a9ef00ca68ef006d0037002d
:1028980014408000e00f5200030032008003eb0078
:1028a800948f13006700350074c0b3000002fd0068
:1028b80044e8b7000002fd00568020001643780067
:1028c8000683fb006780200097437800c83bdd0043
:1028d800060278000702720076802000164378000e
:1028e8000683fb008780200097437800c83bdd0003
:1028f80086027800878272000002fd0045e8b70072
:102908000002fd004823de000003fd0046e8b70092
:102918000003fd008002fd0047e8b7008002fd00cb
:10292800482ade000002fd0048e8b7000002fd006a
:1029380094802000144278000002fd0049e8b700a6
:102948000002fd00e14f5200300036000044eb0069
:102958004a842000f90f20000880fb0001002000b5
:1029680056802000164378000683fb00678020000d
:1029780097437800c83bdd00060278000702720022
:1029880076802000164378000683fb0087802000ad
:1029980097437800c83bdd00860278008782720082
:1029a8000000420081804a0080fe07000881fb0089
:1029b80096802000164378000683fb000603d100aa
:1029c8008683fb00870151000302b0008381410028
:1029d8008301450089496000c805de009b419800d5
:1029e80081826400870351001702b0008783430087
:1029f8008703450089cb6200482ade00944398008b
:102a080008c4e800884f5300d3ff3e0003c4b30056
:102a18004284200011c0b300014078001afb07006f
:102a280010408800ca68ef00060037009424ef00c1
:102a38000082eb00000000000402e900fdff3a00fc
:102a48000000fe004f05be004f04be000000060057
:102a580064942000144278007f426200e14f5200e3
:102a68005d003a00a494200014427800e04f520020
:102a780059003a007494200014427800e64f52003e
:102a88001e003a00949420001442780015c2b30046
:102a9800854f5200040032008542e800854f5200fd
:102aa80016003a000d0037002492200014427800e6
:102ab800e14f520011003a00044d2800c448880034
:102ac80094002000e448880004ccb3000002fd0014
:102ad8001ae9b7000002fd00080037006454280016
:102ae800c4488800d4012000e448880004ccb3001e
:102af8000002fd001ae9b7000002fd0065942000fd
:102b0800954278000546b20004c2b30084cf520053
:102b180031003a0074942000144278000482fb00cb
:102b28000500200062025200e0825a00e90f5200bc
:102b3800e08f5a0028003e000460010009003700b9
:102b48001700370024003700230037002200370021
:102b580021003700200037001f0037000a00370027
:102b68001800370064952000c4488800140020002d
:102b7800e448880014ccb3000002fd001ae9b7004d
:102b88000002fd000000060004c8b300040078003d
:102b98001ae9b70049c9bf0056e9b70000000600a6
:102ba80074952000c448880014002000e448880078
:102bb80014c8b3000002fd001ae9b7000002fd00c6
:102bc8000000060004c8b300040078001ae9b70042
:102bd80048c9bf0057e9b700000006008824ab00c9
:102be80002003200100020007500370005498000ff
:102bf80004022000848f520011003a00d44a800059
:102c0800e10f520003003a0010002000680007009e
:102c18001b003700b5042000850f520003003a005e
:102c28001000200066000700150037006509200025
:102c3800850f5200120036005a29ef0010003700a5
:102c4800d44a8000e10f520003003a00100020002f
:102c5800570007000a00370025032000850f52009f
:102c680003003a0010002000550007000400370058
:102c7800653b2000850f5200010036005a29ef00fd
:102c88005a29ec00000006000000eb0024000700b1
:102c980001fa0700f0fa070004498000ff0f52000c
:102ca800fdff36008824ab00fbff3a00c7fd070094
:102cb800f9ff370034072000840f50000d00320060
:102cc80005003c00e10f500010003200e30f5000f7
:102cd80011003a000f00370044072000840f50000d
:102ce800080032000402e800840f50000a003a008d
:102cf80002003700b9ff070007003700b7ff0700d9
:102d080005003700b5ff0700030037004cfd07003a
:102d1800010037004eff070010c0b3000000060096
:102d2800e00f500011003a0083e0a80010002000d6
:102d38005e0007001000200053000700e04f50001d
:102d480007003a0034082000053a800005026200b6
:102d58000300320083e0a90000180400000000000e
:102d680044a7a800100020002f000700000006005c
:102d78003600f800809fbe00829fbe00849fbe0080
:102d8800869fbe003400f80000002000a0018800e3
:102d980092fc07003400f9004f03be004f02be004a
:102da8004f01be004f00be003600f900004006008b
:102db800e10f500001003a00cca2a9000000060073
:102dc800e10f500001003a00cca2a8000000060064
:102dd800e10f50000a003a00641680004522de0028
:102de8000482ea00610262004522dd00f5fd2f0041
:102df80066168000868262000502720064168800ea
:102e080000000600e10f500005003a007f00400076
:102e1800cc02b6000000e9004f00de00000006000a
:102e28000040eb0000000600e10f500001003a00ee
:082e3800c8a2a9000000060079
:020000040000fa
:102e4000140900004200000000000000000a000019
:102e500020000000000000005609000002000000f1
:102e60000000000000080000140100000000000045
:102e700058090000020000000200000001000000ec
:102e80005a090000020000000000000000000000dd
:020000040000fa
:102e9000e10f500005003a007f004000ca02b60072
:102ea0000000e9004f00de00000006000040eb00db
:102eb00000000600e10f500001003a00c8a2a8007f
:042ec0000000060008
:020000040000fa
:1030000000040400000000009a0404000000000016
:103010009a040400000000009a040400000000006c
:103020009a040400000000009a040400000000005c
:103030009a040400000000009a040400000000004c
:103040009a040400000000009a040400000000003c
:103050009a040400000000009a040400000000002c
:103060009a040400000000009a040400000000001c
:103070009a040400000000009a040400000000000c
:103080009a040400000000009a04040000000000fc
:103090009a040400000000009a04040000000000ec
:1030a0009a040400000000009a04040000000000dc
:1030b0009a040400000000009a04040000000000cc
:1030c0009a040400000000009a04040000000000bc
:1030d0009a040400000000009a04040000000000ac
:1030e0009a040400000000009a040400000000009c
:1030f0009a040400000000009a040400000000008c
:103100009a040400000000009a040400000000007b
:103110009a040400000000009a040400000000006b
:103120009a040400000000009a040400000000005b
:103130009a040400000000009a040400000000004b
:103140009a040400000000009a040400000000003b
:103150009a040400000000009a040400000000002b
:103160009a040400000000009a040400000000001b
:10317000bc160400000000009a04040000000000d7
:020000040000fa
:020000040001f9
:0457f00033ff000083
:020000040000fa
:020000040001f9
:0457f400c0fc0000f5
:020000040000fa
:020000040001f9
:0457f8008e1b000004
:020000040000fa
:020000040001f9
:0457fc00603f00000a
:00000001FF
